:020000040000FA
:020000000428D2
:080008008601890183164030D6
:1000100081000C30850000308600831280308B0018
:10002000892B05169C202A0885049C2005129C20FB
:1000300029088505080005129C2085100510080078
:1000400005120000851405149C2005169C2008004C
:10005000AB0008308F00171064000310AB0D0318BD
:100060000516031C05122A088504000029088505C9
:100070008F0B2C28051683161C30850083122A0846
:100080008504051A4A202908850583160C30850049
:10009000831208001714080008308F00AB01831684
:1000A0001C308500831264002A08850400000310B8
:1000B000AB0D051A2B14290885059C208F0B53289E
:1000C00083160C3085008312051608000516692872
:1000D000051200002A0885049C20290885050516BC
:1000E000080001308C0001308F00922802308F0010
:1000F000902805308F00902832308F0090280530EE
:10010000910084281430910064308F009020910B6E
:1001100084280800260890007920900B8C2808007D
:100120000A308C0081010B1164000B1D94288C0B8C
:1001300092288F0B902808000800AF017C20033024
:10014000C52079200330C52079200330C5207920CF
:100150000230C52076202830B820AF010C30B820FE
:100160000130B8200630B8202030AF0076200800DB
:100170008D000230900064000D08F0399200120EDC
:10018000C5208D0E900BBB28080092003F39171A2E
:100190004038860000002F078604000010388604CF
:1001A0000000EF398605712008008030D828C03063
:1001B00094007120AF0114081307B8202030AF005D
:1001C000080096000B309300D520EC2896000330F1
:1001D0009300D520EC289600F520003E0319080076
:1001E000B820960A0319950AEC2815088A00160803
:1001F000820052344534503445345434203445342C
:100200004534503420342034763431342E34313473
:1002100031340034203464346534763440347334FB
:10022000683469346234623479342E34663472341A
:1002300000343234343458342034203420342034E0
:10024000233420343E340034433448344F3449346A
:100250005834203420342F342034203420342034B7
:10026000203420344F344B340034503452344F3423
:1002700047342034003456344534523449344634FB
:10028000003421344E34413443344B3400344F3441
:100290004B3420343A342934003421344534523438
:1002A00052342034003452344534503452344F34B4
:1002B000473420342F3420345334553449345634A1
:1002C00041344E3454340034503452344F34473473
:1002D0002034203420342F3420342034203420346F
:1002E00049344E3449345434003420345034523478
:1002F0004F34473420345434453452344D34493427
:100300004E344534453421342034003420342034F4
:10031000203420342034203420342034203420343D
:10032000203420342034203420342034003421344C
:10033000443441345434413400343334323420347E
:1003400000343634343420340034363435342034F8
:1003500000343134323438340034323435343634C5
:10036000003435343134323400349301D520003038
:100370009500F930EB20D720013095000A30EB20B2
:100380000800AD209301D520013095001930EB20F5
:10039000D720013095002430EB2008009301D720AE
:1003A000013095006430EB200800013095003530B5
:1003B000E1209301D7200800013095003B30E12077
:1003C0000800013095004130E1209301D720013031
:1003D00095005330EB200800013095009730E12064
:1003E000E5290800013095004D30E120FB2901305E
:1003F00095004730E1209301D720013095007530FA
:10040000EB2008009301D720013095008630EB20C7
:100410009301D7200800013095009D30E6200800A8
:1004200001309500A130E620080001309500A5308C
:10043000E620080001309500A930E62008000130D0
:100440009500AD30E620080001309500B130E6207F
:1004500008000B229B0140309F003F309D00103070
:10046000A1000130A2000430A4000830A6006823D7
:100470007C206400051D3F2A851D0800392A1022B2
:1004800020309F000130A6009B01FF309D002030EE
:10049000A1000230A2001030A40068237C20640078
:1004A000051D552A851D08004F2A152240309F0042
:1004B0007F309D000830A400A60068237C206400E3
:1004C000051D652A851D08005F2A1A220130A60035
:1004D0009B01FF309D004030A1000430A20010308D
:1004E000A40068237C206400051D792A851D08006E
:1004F000732A1F2201309B00FF309D008030A10035
:100500000830A2002030A40068237C206400051D70
:100510008C2A851D0800862A242280309F00003006
:10052000A1001030A20068237C206400051D292A48
:10053000851D0800952AFD30A9000230AA00080098
:10054000FE30A9000130AA000800061717162D0872
:10055000AE006F2319089A0082231B089C001D0817
:100560009E00A701A8012408A5000222D5211F088A
:10057000A0001B209B22A030282027082820280824
:1005800028201120A13028204C202B088E00A022EA
:10059000180828202708282028082820D62A6400A0
:1005A0009B2268204C202B088E00A0220E082820B9
:1005B0001718F32AA80FDD2AA70AA00BCF2A642355
:1005C000A50BE62AFF30B8202408A5008A200130B8
:1005D00003109E020318B72A013003109C0203186F
:1005E000B72A1F2BFD2A66202020E1216823640002
:1005F000051DAC2A851D002BF72A2C08AE056F239C
:100600000314AC0D9718072B06171716132B171981
:10061000112B18080311A63C031D042B9E309800D3
:10062000171506131712023098079A0BAC2AF721F8
:1006300003112E08003C031DF2217F209C2B220871
:10064000A300DC21A701A80102229B221B20A030CD
:10065000282027082820280828201120A130282019
:100660004C202B088E00A0221808282027082820BC
:10067000280828201120180801382820472B64005A
:100680009B2268204C202B088E00A02268204C2042
:1006900003110E082B02031D582BA80F3F2BA70A8E
:1006A0005C2B270803112102031D3F2B6323F22A31
:1006B0006323EC216823F72AA30B512BFF30B820CA
:1006C0002208A300512B66209B22662020200800D0
:1006D0007C206400051D692B851D692B080086138D
:1006E00008308F002E088D00640003108D0C061357
:1006F000031806178617000086138F0B742B08004B
:1007000019089A0008309300D5201A08303EB82006
:1007100008009701AE016F231F3085009D20B52191
:100720008220051DAB2B851DB02B013099000130B7
:10073000AD00C12180232922171117128023FE301A
:10074000AC00CE21A030980068236400051DA52AC6
:10075000851D992BA52B043099000F30AD00992BE6
:0C07600008309900FF30AD009714992B71
:02400E00F63F7B
:00000001FF
